:100000008A010328592983120313860185010630CA
:1000100083169F001F308500860183120313050895
:100020001039003C03191C28050886000A30F1002D
:1000300002208A110A125829F30108307302013094
:1000400003180301003C03196D2883120313860172
:100050007308F000003C031D2F2806146628700862
:10006000013C031D37288312031386146628700889
:10007000023C031D3F2883120313061566287008EF
:10008000033C031D47288312031386156628700856
:10009000043C031D4F2883120313061666287008BC
:1000A000053C031D57288312031386166628700823
:1000B000063C031D5F288312031306176628700889
:1000C000073C031D6628831203138617FF30F100D7
:1000D00002208A110A12F30A1D28831203138601D3
:1000E000F30108307302013003180301003C0319C7
:1000F000C0287308F000003C031D822883120313FC
:100100000614B9287008013C031D8A2883120313C2
:100110008614B9287008023C031D92288312031329
:100120000615B9287008033C031D9A28831203138F
:100130008615B9287008043C031DA22883120313F6
:100140000616B9287008053C031DAA28831203135C
:100150008616B9287008063C031DB22883120313C3
:100160000617B9287008073C031DB928831203132A
:100170008617FF30F10002208A110A12F30A712853
:10018000831203138601FF30F10002208A110A1244
:100190003F30831203138600FF30F10002208A11E2
:1001A0000A120630831203138600FF30F10002208A
:1001B0008A110A125B30831203138600FF30F100AC
:1001C00002208A110A124F30831203138600FF3077
:1001D000F10002208A110A1266308312031386008E
:1001E000FF30F10002208A110A126D3083120313CE
:1001F0008600FF30F10002208A110A127D3083123E
:1002000003138600FF30F10002208A110A12073022
:10021000831203138600FF30F10002208A110A12B4
:100220007F30831203138600FF30F10002208A1111
:100230000A126F30831203138600FF30F100022090
:100240008A110A127730831203138600FF30F100FF
:1002500002208A110A127C30831203138600FF30B9
:10026000F10002208A110A1239308312031386002A
:10027000FF30F10002208A110A125E30831203134C
:100280008600FF30F10002208A110A1279308312B1
:1002900003138600FF30F10002208A110A12713028
:1002A000831203138600FF30F10002208A110A1224
:1002B0000D288E30F2000000000000000000000059
:1002C0000000F20B5D290000F10B59290000080025
:00000001FF
